:020000040000FA
:060000005EEF12F0120099
:020006001200E6
:0600080028EF02F01200D7
:02000E000100EF
:0C001000EE24000000010000E0000000F1
:04001C000F0E93161A
:10002000811665D9939493968194819660D90F0E29
:100030008114816E300E8110816E2BD858D90F0E2D
:100040008116300E811225D852D90F0E8116300E2E
:1000500081129DD91ED870D90F0E811698D9818A28
:1000600096D917D8280EE66E19D8E552080EE66E16
:1000700015D8E552010EE66E11D8E552060EE66E71
:100080000DD8E5520C0EE66E09D8E55280D900D0A5
:10009000120081867CD98196C1EF01F0D9CFE6FFAD
:1000A000E1CFD9FF74D9819481960F0E8116FE0E8F
:1000B000DBCF14F0F00E1414811269D9EADF0F0EB1
:1000C0008116FE0EDB50146E156A040ED89014369D
:1000D0001536E804FBE1F00E1414811258D9D9DF6B
:1000E00000D0E552E7CFD9FF1200D9CFE6FFE1CF2C
:1000F000D9FF4DD9818481960F0E8116FE0EDBCF7C
:1001000014F0156A14BE1568F00E1414811281865D
:100110003ED981960F0E8116FE0EDBCF14F0156AC4
:1001200014BE1568040ED89014361536E804FBE1A9
:10013000F00E1414811281862AD9819600D0E552DE
:10014000E7CFD9FF1200D9CFE6FFE1CFD9FFFD0EEF
:10015000DBCFF6FFFE0EDBCFF7FF0800F5CF14F084
:10016000156A14BE15681450151016E0FD0EDBCF8D
:10017000F6FFFE0EDBCFF7FF0800F5CF14F0156A8F
:1001800014BE15681450E66EB0DFE552FD0EDB2A92
:10019000FE0E01E3DB2ADBD700D0E552E7CFD9FF23
:1001A0001200D9CFE6FFE1CFD9FFFD0EDBCFE9FF8B
:1001B000FE0EDBCFEAFFEFCF14F0156A14BE156810
:1001C0001450151015E0FD0EDBCFE9FFFE0EDBCF5E
:1001D000EAFFEFCF14F0156A14BE15681450E66EEE
:1001E00084DFE552FD0EDB2AFE0E01E3DB2ADDD7BC
:1001F00000D0E552E7CFD9FF1200D9CFE6FFE1CF1B
:10020000D9FFE652FE0EDBCF14F0156A14BE156856
:10021000010E141801E1155009E1FD0EDBCF14F0B9
:10022000156A14BE1568800E1424DF6EFE0EDBCF37
:1002300014F0156A14BE1568020E141801E1155069
:1002400009E1FD0EDBCF14F0156A14BE1568C00E6F
:100250001424DF6EDFCF14F0156A14BE1568145035
:10026000E66E1CDFE552E552E552E7CFD9FF1200FA
:10027000D9CFE6FFE1CFD9FF020EE126E66AFE0EF6
:10028000DBCF14F0156A14BE15681450E66EB5DFA6
:10029000E552E552DE6ADD6ADECF14F0DDCF15F0FF
:1002A000D890155004E6100E145C000E155809E2A3
:1002B000200EE66E1ADFE552DF2A010E01E3DB2A8B
:1002C000EBD7E66AFE0EDBCF14F0156A14BE156894
:1002D0001450E66E92DFE552E552020EE15C02E256
:1002E000E16AE552E16EE552E7CFD9FF1200D9CFBE
:1002F000E6FFE1CFD9FF020EE126DE6ADD6ADECF3E
:1003000014F0DDCF15F0D890155004E6100E145CF3
:10031000270E155806E20000DF2A010E01E3DB2A52
:10032000EED700D0020EE15C02E2E16AE552E16E36
:10033000E552E7CFD9FF1200D9CFE6FFE1CFD9FFD1
:10034000020EE126DE6ADD6ADECF14F0DDCF15F0A5
:10035000D890155004E6C40E145C090E155806E238
:100360000000DF2A010E01E3DB2AEED700D0020EE7
:10037000E15C02E2E16AE552E16EE552E7CFD9FFC6
:100380001200000000000000000000001200D9CFA1
:10039000E6FFE1CFD9FF020EE126DE6ADD6ADECF9D
:1003A00014F0DDCF15F0D890155004E6E80E145C7B
:1003B000030E155806E20000DF2A010E01E3DB2AD6
:1003C000EED700D0020EE15C02E2E16AE552E16E96
:1003D000E552E7CFD9FF1200D9CFE6FFE1CFD9FF31
:1003E00081940F0E8116FE0EDB50146E156A400EBE
:1003F0001412000E1512F00E14148112C2DF49DE21
:100400000F0E8116FE0EDB50146E156A040ED89086
:1004100014361536E804FBE1F00E14148112B1DF36
:1004200038DE00D0E552E7CFD9FF1200000000000F
:1004300000000000000000000000000000000000BC
:10044000000000000000000000000000000012009A
:10045000DACFE4FFE2CFDAFFE6529E50010B1C6ECA
:100460001D6A010E1C1801E11D5007E10001752BEA
:10047000000E7623772378239E90E552E5CFDAFFAE
:100480001100D9CFE6FFE1CFD9FFFB0EDBCF05F09E
:10049000FC0EDBCF06F0FD0EDBCF07F0FE0EDBCF50
:1004A00008F00834000E081809E6D880000E05543C
:1004B000000E0654000E0754000E08540CE2D950EA
:1004C000FB0FE96EFF0EDA20EA6EEE06000EEE5A22
:1004D000EE5AEE5ADAD7E552E7CFD9FF1200948EE2
:1004E000949C400EAF6EAC8AAC84AC98AC9CAB8E46
:1004F000AB9CAB889E989E9A9D9AF29EF29C1200AD
:10050000D9CFE6FFE1CFD9FFE6520001AA51A819E1
:1005100002E1AB51A91901E1F8D7A8C0E9FFA9C0D0
:10052000EAFFA82B000EA923EFCF14F0156A14BE22
:1005300015681450DF6EDE0EA85D010EA95904E3A4
:100540008E0EA86F010EA96FDF5000D0E552E55264
:10055000E7CFD9FF1200D9CFE6FFE1CFD9FF020ED6
:10056000E126DE6ADD6AAC50020B01E0010E146E7A
:10057000156A1450151017E1DF2A010E01E3DB2A7A
:10058000DECF14F0DDCF15F0166A1634000E161803
:1005900007E6D880E80E1454FD0E1554000E1654CC
:1005A00001E201D0E0D7FE0EDB50AD6E9E50100B85
:1005B00001E0010E146E156A1450151001E1F6D712
:1005C000020EE15C02E2E16AE552E16EE552E7CF3C
:1005D000D9FF1200D9CFE6FFE1CFD9FF030EE12604
:1005E000FD0EDBCFDEFFDBCFDDFF8ADFE76E020E25
:1005F000E7CFDBFFDBCF14F0156A14BE1568FC0EE5
:10060000DBCF16F0176A16BE17681650141802E1F1
:100610001750151812E0020EDBCF14F0156A14BE45
:100620001568FD0EDBCFE9FFDB2AFE0EDBCFEAFF0C
:1006300001E3DB2A14C0EFFFD8D7FD0EDBCFE9FFC3
:10064000FE0EDBCFEAFFEF6ADECF14F0DDCF15F050
:1006500014C0F3FF15C0F4FF030EE15C03E200D009
:10066000E16AE552E16EE552E7CFD9FF1200D9CF3A
:10067000E6FFE1CFD9FF020EE126DE6ADD6AFD0E5C
:10068000DBCFE9FFFE0EDBCFEAFFEF50146E156AF9
:100690001450151014E0FD0EDBCFE9FFFE0EDBCF8A
:1006A000EAFFEF50E66E57DFE552DF2A010E01E365
:1006B000DB2AFD0EDB2AFE0E01E3DB2AE0D7010E6A
:1006C000F36EF46A020EE15C03E200D0E16AE552E7
:1006D000E16EE552E7CFD9FF12000D0EE66E3BDF6B
:1006E000E5520A0EE66E37DFE5521200D9CFE6FF7B
:1006F000E1CFD9FF0A0EE12600017D0E9B6F010EAE
:100700009C6FFC0EDBCF14F0156A14BE156815340F
:1007100004E214500108000E155401E2F9D0FC0E59
:10072000DBCF14F0156A14BE15681450151028E1BB
:10073000FD0EDBCF14F0FE0EDBCF15F0060E14C05D
:10074000DBFF070E15C0DBFF080EDB6A090EDB6A54
:100750009BC0E6FF9CC0E6FFD950060FE96EDACFDA
:10076000EAFFEECFE6FFEECFE6FFEECFE6FFEFCFFC
:10077000E6FF92EC0FF0146E060EE15E145010D0FE
:100780009BC0E6FF9CC0E6FFFD0EDBCFE6FFFE0E42
:10079000DBCFE6FFF8EC0EF0E552E552E552E5520C
:1007A00000016051400B01E0010E146E156A1450F7
:1007B000151001E191D07D0EE66E010EE66ED2ECD1
:1007C00011F0E552E552020EF3CFDBFF030EF4CF3A
:1007D000DBFFDE6ADD6ADECF14F0DDCF15F0020E3E
:1007E000DBCF16F0030EDBCF17F01650145C17505A
:1007F000155831E2020EDBCF16F0030EDBCF17F0F7
:10080000DE50165CE96EDD501758EA6EE906000E00
:10081000EA5A7D0EE926010EEA22EF50E66EFC0E42
:10082000DBCF14F0156A14BE1568040E1426000EF2
:100830001522DE50145CE96EDD501558EA6E7D0E0F
:10084000E926010EEA22E552E750EF6EDF2A010E9B
:1008500001E3DB2AC0D7DE6ADD6ADECF14F0DDCF2C
:1008600015F0FC0EDBCF18F0196A18BE1968050EDA
:100870001826000E1922020EDB50185C166E030EAD
:10088000DB501958176E1650145C1750155824E297
:1008900000016051100B01E0010E146E156A145036
:1008A00015100BE0DECFE9FFDDCFEAFF7D0EE92674
:1008B000010EEA22300EEF6E0AD0DECFE9FFDDCF67
:1008C000EAFF7D0EE926010EEA22200EEF6EDF2AF6
:1008D000010E01E3DB2AC1D7FC0EDBCFE9FFEA6A98
:1008E000E9BEEA68050EE926000EEA227D0EE92639
:1008F000010EEA22EF6A9BC0E6FF9CC0E6FFB7DE6E
:10090000E552E552020EF3CFDBFF030EF4CFDBFF1F
:100910000A0EE15C02E2E16AE552E16EE552E7CFE0
:10092000D9FF1200D9CFE6FFE1CFD9FF0E0EE126A5
:10093000F90EDBCFDEFFDBCFDDFFF80EDBCF16F0ED
:10094000176A16BE1768173404E216500008000E26
:10095000175404E3070E146E156A1BD0F80EDBCF94
:1009600018F0196A18BE1968193404E218501608EC
:10097000000E195404E2170E146E156A0AD0F80E10
:10098000DBCF14F0156A14BE1568010E1426000E94
:100990001522080E14C0DBFF090E15C0DBFF020E86
:1009A000DB6A030EDB6AFB0EDBCF14F0FC0EDBCF41
:1009B00015F0FD0EDBCF16F0FE0EDBCF17F00A6A46
:1009C0000B6A0C6A0D6A14C005F015C006F016C05B
:1009D00007F017C008F014EC0EF0010A33E1F90E2D
:1009E000DBCFE9FFDB2AFA0EDBCFEAFF01E3DB2AEC
:1009F0002D0EEF6EFB0EDBCF14F0FC0EDBCF15F0EF
:100A0000FD0EDBCF16F0FE0EDBCF17F00A6A0B6A85
:100A1000800E0C6EBF0E0D6E14C005F015C006F0F2
:100A200016C007F017C008F06FEC0DF0FB0E05C004
:100A3000DBFFFC0E06C0DBFFFD0E07C0DBFFFE0E7A
:100A400008C0DBFFFB0EDBCF14F0FC0EDBCF15F094
:100A5000FD0EDBCF16F0FE0EDBCF17F00A6A0B6A35
:100A60000C6A0D6A14C005F015C006F016C007F038
:100A700017C008F00BEC0EF0010A4AE1FB0EDBCFC9
:100A800014F0FC0EDBCF15F0FD0EDBCF16F0FE0EE2
:100A9000DBCF17F00A6A0B6A800E0C6E3F0E0D6EEC
:100AA00014C005F015C006F016C007F017C008F016
:100AB00014EC0EF0010A2CE1146A156A200E166E71
:100AC000410E176ED950FB0FE96EFF0EDA20EA6E69
:100AD000EECF05F0EECF06F0EECF07F0EFCF08F047
:100AE00014C00AF015C00BF016C00CF017C00DF0C2
:100AF0006FEC0DF008C0EDFF07C0EDFF06C0EDFF85
:100B000005C0EFFF020EDB06030E01E2DB06B6D7DF
:100B1000FB0EDBCF14F0FC0EDBCF15F0FD0EDBCFB0
:100B200016F0FE0EDBCF17F00A6A0B6A200E0C6E71
:100B3000410E0D6E14C005F015C006F016C007F08A
:100B400017C008F014EC0EF0010A2EE0FB0EDBCF0C
:100B500014F0FC0EDBCF15F0FD0EDBCF16F0FE0E11
:100B6000DBCF17F00A6A0B6A200E0C6E410E0D6E79
:100B700014C005F015C006F016C007F017C008F045
:100B80001CEC0DF0FB0E05C0DBFFFC0E06C0DBFF0E
:100B9000FD0E07C0DBFFFE0E08C0DBFF020EDB2AE6
:100BA000030E01E3DB2AB4D7020EDBCF14F0030EF1
:100BB000DBCF15F0D950080FE96EDACFEAFF1450F9
:100BC000EE261550ED22010EF36E040EF3CFDBFF7F
:100BD000050EDB6A040EDBCF06F0050EDBCF07F057
:100BE00057EC0CF00A0E05C0DBFF0B0E06C0DBFF56
:100BF0000C0E07C0DBFF0D0E08C0DBFF040EDBCFC1
:100C000014F0050EDBCF15F0080EDBCF16F0090E41
:100C1000DBCF17F015501718E8AE02D0173404D008
:100C20001650145C175015582EE20A0EDBCF14F044
:100C30000B0EDBCF15F00C0EDBCF16F00D0EDBCF5D
:100C400017F00A6A0B6A200E0C6E410E0D6E14C06E
:100C500005F015C006F016C007F017C008F01CEC30
:100C60000DF00A0E05C0DBFF0B0E06C0DBFF0C0EFD
:100C700007C0DBFF0D0E08C0DBFF040EDB2A050EEC
:100C800001E3DB2ABBD70A0EDBCF18F00B0EDBCF5C
:100C900019F00C0EDBCF1AF00D0EDBCF1BF00A6A39
:100CA0000B6A0C6A400E0D6E18C005F019C006F0F4
:100CB0001AC007F01BC008F01CEC0DF005C014F0C2
:100CC00006C015F007C016F008C017F0D950FB0F8A
:100CD000E96EFF0EDA20EA6EEECF05F0EECF06F0F9
:100CE000EECF07F0EFCF08F014C00AF015C00BF0FC
:100CF00016C00CF017C00DF086EC0CF008C0EDFF2C
:100D000007C0EDFF06C0EDFF05C0EFFFFB0EDBCF18
:100D100014F0FC0EDBCF15F0FD0EDBCF16F0FE0E4F
:100D2000DBCF17F00A6A0B6A200E0C6E410E0D6EB7
:100D300014C005F015C006F016C007F017C008F083
:100D400014EC0EF0010A13E0FB0EDB6AFC0EDB6A0A
:100D5000800EF36EFD0EF3CFDBFF3F0EF36EFE0E43
:100D6000F3CFDBFF020EDB2A030E01E3DB2A020EC8
:100D7000DBCF14F0030EDBCF15F00001800E15144D
:100D80005FE0F90EDBCFE9FFDB2AFA0EDBCFEAFFEB
:100D900001E3DB2A300EEF6EF90EDBCFE9FFDB2A31
:100DA000FA0EDBCFEAFF01E3DB2A2C0EEF6E080E12
:100DB000DBCF14F0090EDBCF15F0800E151414E014
:100DC000020EDBCF16F0030EDBCF17F0080EDB5060
:100DD000165C146E090EDB501758156E020E14C007
:100DE000DBFF030E15C0DBFF040EDB68050EDB68BE
:100DF000040EDBCF14F0050EDBCF15F0020EDBCFB7
:100E000016F0030EDBCF17F017501518E8AE02D01E
:100E1000153404D01450165C1550175811E2F90E11
:100E2000DBCFE9FFDB2AFA0EDBCFEAFF01E3DB2AA7
:100E3000300EEF6E040EDB06050E01E2DB06D8D79E
:100E4000040EDB6A050EDB6A040EDBCF14F0050E20
:100E5000DBCF15F0080EDBCF16F0090EDBCF17F055
:100E600015501718E8AE02D0173404D01650145C91
:100E70001750155801E3ACD0FB0EDBCF05F0FC0E8C
:100E8000DBCF06F0FD0EDBCF07F0FE0EDBCF08F068
:100E9000DCEC0DF0060E06C0DBFF070E07C0DBFF23
:100EA000300EE76E060EDBCF14F0070EDBCF15F029
:100EB000E7501426000E1522F90EDBCFE9FFDB2ADE
:100EC000FA0EDBCFEAFF01E3DB2A14C0EFFF040ECA
:100ED000DBCF14F0050EDBCF15F0020EDB5014183B
:100EE00003E1030EDB5015180BE1F90EDBCFE9FF30
:100EF000DB2AFA0EDBCFEAFF01E3DB2A2C0EEF6ED2
:100F0000060EDBCF06F0070EDBCF07F057EC0CF038
:100F10000A0E05C0DBFF0B0E06C0DBFF0C0E07C080
:100F2000DBFF0D0E08C0DBFF05C014F006C015F096
:100F300007C016F008C017F0D950FB0FE96EFF0E7E
:100F4000DA20EA6EEECF05F0EECF06F0EECF07F036
:100F5000EFCF08F014C00AF015C00BF016C00CF06B
:100F600017C00DF085EC0CF008C0EDFF07C0EDFFD9
:100F700006C0EDFF05C0EFFF146A156A200E166E5D
:100F8000410E176ED950FB0FE96EFF0EDA20EA6EA4
:100F9000EECF05F0EECF06F0EECF07F0EFCF08F082
:100FA00014C00AF015C00BF016C00CF017C00DF0FD
:100FB0006FEC0DF008C0EDFF07C0EDFF06C0EDFFC0
:100FC00005C0EFFF040EDB2A050E01E3DB2A3CD748
:100FD000F90EDBCFE9FFFA0EDBCFEAFFEF6A0E0E68
:100FE000E15C02E2E16AE552E16EE552E7CFD9FF4A
:100FF00012008168936A9380939293949396939846
:10100000939A939C938E816AC26A070EC16E170EE3
:10101000926E826894809482948494969498949A20
:10102000949C948E1200E5DF89966FEC02F0AD6A15
:10103000AC50020B01E0010E146E156A145015102D
:1010400001E1F6D7200EE66E37EC12F0E5520C0EF9
:10105000E66EABEC02F0E552400EE66E0D0EE66E6B
:10106000030EE66EE66A41EC02F0E552E552E55207
:10107000E5526DEC03F00001240E996F010E9A6F9A
:10108000010E00016B6F6C6B0001050E6B5D000EB5
:101090006C5934E26BC0E9FF6CC0EAFF010ED890D6
:1010A000E936EA36E806FBE1000EE926010EEA22FF
:1010B000EECF14F0EFCF15F0166A14C0E6FF15C09E
:1010C000E6FF16C0E6FF99C0E6FF9AC0E6FFB9EC5E
:1010D00011F0176E050EE15E175099C0E6FF9AC039
:1010E000E6FF37EC03F0E552E552F3CF6FF0F4CFB3
:1010F00070F000016B2B000E6C23C6D70001608FCF
:101100000EEC00F0010EE66E4EEC00F0E552880E9B
:10111000E66E130EE66EE66AE66A41EC02F0E55210
:10112000E552E552E55200016B6B6C6B0001050E58
:101130006B5D000E6C592DE2800EE66E4EEC00F0F9
:10114000E5526BC0E9FF6CC0EAFF010ED890E936AA
:10115000EA36E806FBE10E0EE926010EEA22EECFA2
:10116000E6FFEFCFE6FFA3EC00F0E552E552F00E0C
:10117000E66E490EE66E020EE66EE66A41EC02F09D
:10118000E552E552E552E55200016B2B000E6C234F
:10119000CDD7D56AD59ED59CD59AD598D584D582FC
:1011A000D590D5966A0EE66E670EE66E1BEC12F0D1
:1011B000E552E552F294F29ACD6ACD8ECD9ACD9851
:1011C000CD96CD84CD82CD909F80000EE66EE66AEE
:1011D000FFEC11F0E552E5529E90BD6AF28C9D90B5
:1011E000F29EF29C8050040B01E0010E146E156A11
:1011F000010E141801E1155026E1010E0001796F6E
:101200007A6B0AC114F00BC115F0166A14C0E6FF20
:1012100015C0E6FF16C0E6FF99C0E6FF9AC0E6FFDC
:10122000B9EC11F0176E050EE15E175099C0E6FF9C
:101230009AC0E6FF37EC03F0E552E552F3CF6FF0CA
:10124000F4CF70F025D0040E0001796F7A6B0CC1D9
:1012500014F00DC115F0166A14C0E6FF15C0E6FFC4
:1012600016C0E6FF99C0E6FF9AC0E6FFB9EC11F0A0
:10127000176E050EE15E175099C0E6FF9AC0E6FFB3
:1012800037EC03F0E552E552F3CF6FF0F4CF70F096
:101290006DEC03F00001676B686B0101DF6B00010F
:1012A000756B766B776B786B00017B6B7C6B0001E9
:1012B0007F6B806B00017D6B7E6BCD906A0EE66E5E
:1012C000670EE66E1BEC12F0E552E552000EE66E7C
:1012D000E66AFFEC11F0E552E5529E9AF294D08E48
:1012E0009E908050040B01E0010E146E156A010EF1
:1012F000141801E1155005E1010E0001796F7A6BB8
:1013000004D0040E0001796F7A6BF29CF28E010119
:10131000226B236BF29AF2949D80D58E8986CD80C4
:10132000F250040B01E0010E146E156A14501510F2
:1013300001E1F6D70F0EE66E6CEC12F0E55201D02B
:1013400001D000000000010E010122250101226FE1
:10135000000E010123210101236FF2946A0EE66E53
:10136000670EE66E1BEC12F0E552E5520001795172
:101370000101225D00017A5101012359D1E38996CF
:10138000D59ECD90E0EC11F0F3CF7BF0F4CF7CF064
:10139000F294F29AF29E7BC006F07CC007F055EC06
:1013A0000CF005C08BF006C08CF007C08DF008C0B3
:1013B0008EF075C004F076C005F077C006F078C0F6
:1013C00007F06AEC0CF005C014F006C015F007C079
:1013D00016F008C017F00A6A0B6A800E0C6E470EF2
:1013E0000D6E14C005F015C006F016C007F017C04A
:1013F00008F06FEC0DF005C083F006C084F007C064
:1014000085F008C086F083C00AF084C00BF085C068
:101410000CF086C00DF08BC005F08CC006F08DC0BE
:1014200007F08EC008F086EC0CF005C087F006C00F
:1014300088F007C089F008C08AF0800EE66E4EEC96
:1014400000F0E5520001240E996F010E9A6F805052
:10145000040B01E0010E146E156A1450151036E1EC
:101460000A6A0B6A800E0C6E400E0D6E87C005F086
:1014700088C006F089C007F08AC008F01CEC0DF0A7
:1014800005C087F006C088F007C089F008C08AF060
:10149000010EE66E99C0E6FF9AC0E6FF87C0E6FF40
:1014A00088C0E6FF89C0E6FF8AC0E6FF92EC04F040
:1014B000146E070EE15E1450340EE66E75EC00F00B
:1014C000E552080E0001736F746B37D0310EE66E73
:1014D00075EC00F0E552010EE66E99C0E6FF9AC089
:1014E000E6FF87C0E6FF88C0E6FF89C0E6FF8AC046
:1014F000E6FF92EC04F0146E070EE15E145099C002
:10150000E6FF9AC0E6FFD2EC11F0E552E552F3CFC8
:101510006FF0F4CF70F00001020E6F5F000E705B91
:10152000240E00016F25E96E010E00017021EA6EA4
:10153000EF6A060E0001736F746B530EE66E75EC66
:1015400000F0E552460EE66EABEC02F0E552720E8C
:10155000E66EABEC02F0E552650EE66EABEC02F027
:10156000E552710EE66EABEC02F0E5523D0EE66E12
:10157000ABEC02F0E552200EE66EABEC02F0E55269
:1015800099C0E6FF9AC0E6FFD2EC11F0E552E552B1
:10159000F3CF6FF0F4CF70F00001716B726B00014C
:1015A0006D6B6E6B00016F510001735D0001705136
:1015B000000174593BE200016F510001735D0001AD
:1015C00070510001745924E2240E00016D25E96E6A
:1015D000010E00016E21EA6EEFCF14F0156A14BE01
:1015E00015687D0E00017125E96E010E0001722162
:1015F000EA6E14C0EFFF00016F07000E705B000180
:101600006D2B000E6E230001712B000E7223D3D7B9
:101610007D0E00017125E96E010E00017221EA6E56
:101620002E0EEF6E0001712B000E722373C073F04B
:1016300074C074F00001030E735F000E745B000150
:101640006F510001735D00017051000174593BE25C
:1016500000016F510001735D000170510001745968
:1016600024E2240E00016D25E96E010E00016E21B9
:10167000EA6EEFCF14F0156A14BE15687D0E0001F6
:101680007125E96E010E00017221EA6E14C0EFFFB0
:1016900000016F07000E705B00016D2B000E6E23C2
:1016A0000001712B000E7223D3D77D0E000171252E
:1016B000E96E010E00017221EA6E2E0EEF6E00013E
:1016C000712B000E722373C073F074C074F00001AC
:1016D000030E735F000E745B00016F510001735DB8
:1016E00000017051000174592BE20001000ED880F6
:1016F0006F55000E705524E2240E00016D25E96E31
:10170000010E00016E21EA6EEFCF14F0156A14BECF
:1017100015687D0E00017125E96E010E0001722130
:10172000EA6E14C0EFFF00016F07000E705B00014E
:101730006D2B000E6E230001712B000E7223D5D786
:101740007D0E00017125E96E010E00017221EA6E25
:10175000480EEF6E0001712B000E72237D0E00010A
:101760007125E96E010E00017221EA6E7A0EEF6EAC
:101770000001712B000E72237D0E00017125E96EB0
:10178000010E00017221EA6EEF6A7D0EE66E010E17
:10179000E66ED2EC11F0E552E552F3CF6FF0F4CFE4
:1017A00070F000010E0E6F5D000E70590AE2200EFF
:1017B000E66E75EC00F0E55200016F2B000E702311
:1017C000F0D77D0EE66E010EE66ED1EC00F0E5522C
:1017D000E5527D0EE66E010EE66E37EC03F0E55243
:1017E000E552F3CF6FF0F4CF70F06DEC03F0000131
:1017F000672B000E68230001090ED8806755000E84
:10180000685551E20001676B686B8050040B01E082
:10181000010E146E156A010E141801E1155022E133
:101820000AC114F00BC115F0166A14C0E6FF15C00A
:10183000E6FF16C0E6FF99C0E6FF9AC0E6FFB9ECE6
:1018400011F0176E050EE15E175099C0E6FF9AC0C1
:10185000E6FF37EC03F0E552E552F3CF6FF0F4CF3B
:1018600070F021D00CC114F00DC115F0166A14C02F
:10187000E6FF15C0E6FF16C0E6FF99C0E6FF9AC076
:10188000E6FFB9EC11F0176E050EE15E175099C036
:10189000E6FF9AC0E6FF37EC03F0E552E552F3CFDE
:0A18A0006FF0F4CF70F0F9D41200DD
:0618AA000F9E08D00F9E06
:1018B00007AE05D0066C071EE86A07220F8E07C028
:1018C00001F006C000F0136A126A8E0E026E036AFF
:1018D0008EEF0EF00F9E0CD00F9E07AE09D0046C59
:1018E000051E061E071EE86A0522062207220F8E25
:1018F00007C001F006C000F005C013F004C012F0EC
:101900009E0E026E036A8EEF0EF00D7E0F6ACAEC19
:101910000EF0E2EC0EF00FB672EF0EF00FA20AD04E
:101920000FAA03D00FBE72EF0EF00FA47EEF0EF0E1
:101930007BEF0EF00FAA05D00FAC7EEF0EF07BEF21
:101940000EF00FA00AD00FA808D00FBE04D00FA42D
:1019500002D087EF0EF08BEF0EF0126A036A0D5083
:10196000085C116E10E305C013F006C000F007C05C
:1019700001F008C010F00AC005F00BC006F00CC062
:1019800007F00F3A09D00AC013F00BC000F00CC0EA
:1019900001F00DC010F0116C0F9E0FBC0F8E10C027
:1019A00002F00FB0BAEF0EF01A0E1160BAEF0EF09F
:1019B000026A086A0FA408D0056C061E071E081EDE
:1019C000E86A0622072208220FAC08D0136C001E1A
:1019D000011E021EE86A002201220222046A11523C
:1019E00007E008340732063205320432112EF9D7E7
:1019F00005501326065000220750012208500222EB
:101A000004C012F00F9E02AE0BD0126C131E001E0B
:101A1000011E021EE86A13220022012202220F8EFA
:101A200002A006D0D8800132003213321232102ABE
:101A300010C002F08EEF0EF00F6ACAEC0EF0E2EC6E
:101A40000EF00FB672EF0EF00FA205D00FBA72EFC4
:101A50000EF079EF0EF00FBA85EF0EF00FA005D063
:101A60000FB872EF0EF085EF0EF00FB879EF0EF0B1
:101A7000036A7F0E0824026EE86A03220D50025E9C
:101A8000E86A035A1A0E106E086A126A136A006A2C
:101A9000016A0A50055E0B50065A0C50075A000E98
:101AA000085A09E70A5005260B5006220C50072257
:101AB000000E082201D0128AD89005360636073665
:101AC0000836D8901236133600360136102EE1D77C
:101AD000075006100510D8A4128A8EEF0EF00F6A78
:101AE000CAEC0EF0E2EC0EF00FB672EF0EF00FA2A1
:101AF00005D00FB872EF0EF079EF0EF00FAA05D0F7
:101B00000FB072EF0EF079EF0EF00FB002D00FA809
:101B100002D085EF0EF0036A0D500824026EE86AC9
:101B200003227E0E025EE86A035A126A136A006A92
:101B3000016A0C500702F4CF01F0F3CF00F00B5014
:101B40000702F3501326F4500022000E01220C501D
:101B50000602F3501326F4500022000E01220A5010
:101B60000702F3501226F4501322000E0022012225
:101B70000B500602F3501226F4501322000E0022DE
:101B800001220C500502F3501226F4501322000ECD
:101B9000002201220A500602F4501226000E1322DF
:101BA000002201220B500502F4501226000E1322CF
:101BB000002201228EEF0EF00F6ACAEC0EF00FB673
:101BC000E6EF0DF00FA20ED00FB405D07F0E076E1A
:101BD000FF0E066E1FD0800E076E066A1BD0076AC6
:101BE000066A18D00FB0FBD78F0E0860EDD77E0EB7
:101BF0000864F5D78E0E085C05E0D89007320632EF
:101C0000082AF8D70FA406D0066C071EE86A072238
:101C100007AEE5D712001DEC0EF00FB6000C0FB0AA
:101C2000000C0FB4000C010C1DEC0EF00FB6000CF4
:101C30000FB0000C0FA4000C010C0F6ACAEC0EF0E0
:101C4000E2EC0EF00FB612000FAE08D00FA004D0D9
:101C50000FA802D00F8012000F9012000D50085CE8
:101C60000BE10C50075C08E10B50065C05E10A50E3
:101C7000055C02E10F801200D8A002D00F8E10D0B8
:101C800008500DC008F00D6E07500CC007F00C6E28
:101C900006500BC006F00B6E05500AC005F00A6E28
:101CA0000D50085C10E0FF0F09E00F900FB403D057
:101CB0000FAE0F8412000FAE0F9412000D2AD890B1
:101CC0000C320B320A320A50055E0B50065A0C5089
:101CD000075A07BEEAD7D890053606360736082ECB
:101CE000F8D7C8D77F0E086EFF0E076E066E056E1A
:101CF00012007F0E0FBEFF0E086E02D07F0E086E20
:101D0000800E076E066A056AF3D70FAE04D0800E08
:101D1000086E076AF7D7086A076AF4D701500010FF
:101D200013101210F8E003BEF0D701BE0CD0025021
:101D30000310EBE0D8901236133600360136020657
:101D4000D8A00306F2D70350D4E10228D2E012AEA5
:101D500011D07F0E121402E113A00CD0132AE86AEE
:101D60000022012207E3D880013200321332022A16
:101D70000228BFE00250C9E013C005F000C006F021
:101D80000134076E0230086E0732089E0FBE088EBF
:101D900078EF0EF00736083602E30F840F7E06E177
:101DA0000F80086A076A066A056A1200082803E0BD
:101DB000D88007321200D890073202E10F82120059
:101DC0000F8612000C360D3602E30F8C0F7E06E1F3
:101DD0000F880D6A0C6A0B6A0A6A12000D2803E06C
:101DE000D8800C321200D8900C32EAE10F8A12002F
:101DF000D9CFE6FFDACFE6FFFA0EE3CFD9FFFB0E2D
:101E0000E3CFDAFFFD0EE35209E72D0EDE6EFC0E86
:101E1000E31EE32AFD0ED8B4E306E31EE652E652C3
:101E2000E652FD0EE124E76EFF0EE220E46EE6527C
:101E3000F70EE3CFE6FFF70EE3CFE6FF68EC0FF017
:101E4000F90EE124E96EFF0EE220EA6E58EC0FF085
:101E50000AE155EC0FF009E158EC0FF008E155EC00
:101E60000FF007E108D063EC0FF05EEC0FF063ECCD
:101E70000FF05EEC0FF063EC0FF0DE6AF90EE12676
:101E8000FF0EE222FF0EE3CFDAFFE552FF0EE3CFB3
:101E9000D9FFE552FC0EE124E96EFF0EE220EA6E66
:101EA000EECFF3FFEFCFF4FF1200EF380F0B12006D
:101EB000EF500F0B02E1EE52D8841200EF380F0BF7
:101EC000300FDE6E1200EE500F0B300FDE6E120080
:101ED000FC0EE3CFE9FFFD0EE3CFEAFF100EE66E46
:101EE000EE6AEE6AEF6AD890FD0EE336FE0EE33638
:101EF000ED36ED36EF36FF0EE30609E089EC0FF024
:101F0000EE5289EC0FF0EE5289EC0FF0EDD7E56E52
:101F10001200030EEF24E8B6EF6E300EEF24E8BE99
:101F2000EF6E000CD9CFE6FFDACFE6FFF80EE3CF75
:101F3000D9FFF90EE3CFDAFFE652E652E652E65257
:101F4000E652FB0EE124E76EFF0EE220E46EE6525D
:101F5000F30EE3CFE6FFF30EE3CFE6FFF30EE3CF9E
:101F6000E6FFF30EE3CFE6FF17EC10F0F50EE124E9
:101F7000E96EFF0EE220EA6E04EC10F019E107ECC6
:101F800010F018E104EC10F017E107EC10F016E186
:101F900004EC10F015E107EC10F014E104EC10F083
:101FA00013E107EC10F012E104EC10F011E112D093
:101FB0000DEC10F012EC10F00DEC10F012EC10F033
:101FC0000DEC10F012EC10F00DEC10F012EC10F023
:101FD0000DEC10F012EC10F0DE6AF50EE126FF0EAB
:101FE000E222FF0EE3CFDAFFE552FF0EE3CFD9FF87
:101FF000E552FA0EE124E96EFF0EE220EA6EEECF22
:10200000F3FFEFCFF4FF1200EF380F0B1200EF5089
:102010000F0B02E1EE52D8841200EF380F0B300F95
:10202000DE6E1200EE500F0B300FDE6E1200FA0E55
:10203000E3CFE9FFFB0EE3CFEAFF200EE66EEE6A88
:10204000EE6AEE6AEE6AEF6AD890FB0EE336FC0E9B
:10205000E336FD0EE336FE0EE336ED36ED36ED36B5
:10206000ED36EF36FF0EE3060FE046EC10F0EE52D1
:1020700046EC10F0EE5246EC10F0EE5246EC10F04A
:10208000EE5246EC10F0E1D7E56E1200030EEF249D
:0E209000E8B6EF6E300EEF24E8BEEF6E000CE7
:02209E000080C0
:1020A00080808080800000C0C0C0C0C0C00000E050
:1020B000E0E0E0E0E00000F0F0F0F0F0F00000F828
:1020C000F8F8F8F8F80000FCFCFCFCFCFC0000FE52
:1020D000FEFEFEFEFE0000FFFFFFFFFFFF00001000
:1020E000181C1E1C1810000103070F070301040E23
:1020F0001F0E0E0E0E0E0E0E0E0E0E1F0E040204FE
:102100000E111F100E0008040E111F100E000804FF
:102110000E010F110F0002050200000000002E2E1C
:102120002E002056657273696F6E20313331303066
:102130003220617665632050494331384632353864
:1021400020200D0A0020506F727420636F6D6D2087
:102150003139323030206F757665727420513D32DE
:10216000304D687A0D0A00204672657175656E63A0
:10217000656D657472652031487A202E2E203130CD
:10218000204D487A0D0A002054696D657231205344
:10219000414E53207072657363616C6572203D20FF
:1021A000636F6D7074657572206427696D70756CEE
:1021B00073696F6E73200D0A002054696D6572306B
:1021C000203D2066656E6574726520646520636FCE
:1021D0006D7074616765202C6261736520312073B6
:1021E00065632061766563205241323D31200D0ADE
:1021F000002054696D657230203D2066656E6574FF
:10220000726520646520636F6D7074616765202C52
:102210006261736520342073656320617665632095
:102220005241323D30200D0A0046726571656E6381
:10223000656D65747265202020003138463235386E
:1022400020513D32304D687A20200067616D6D6508
:102250002031487A2E2E31304D687A0031303025C9
:10226000204D504C41422043313820200076657289
:1022700073696F6E203133313030322020004D656C
:1022800073757220656E2031206F7520347300568F
:1022900069612065746174206465205241322000B8
:1022A000202020202020202020202020202020202E
:1022B000002020202020202020202020202020203E
:1022C00020007061756C666A756A6F2E667265654E
:0322D0002E660077
:0C22D4000E0EF66E000EF76E000EF86E97
:1022E00001010900F550E56F0900F550E66F03E1C3
:1022F000E56701D03DD00900F550E06F0900F550C9
:10230000E16F0900F550E26F09000900F550E96E30
:102310000900F550EA6E090009000900F550E36F65
:102320000900F550E46F09000900F6CFE7F1F7CF97
:10233000E8F1F8CFE9F1E0C1F6FFE1C1F7FFE2C152
:10234000F8FF0101E35302E1E45307E00900F5500F
:10235000EE6EE307F8E2E407F9D7E7C1F6FFE8C15C
:10236000F7FFE9C1F8FF0101E507000EE65BBFD703
:02237000120059
:0E237200FB0EE3CFF6FFFC0EE3CFF7FFFD0EF0
:10238000E3CFF8FFFE0EE3CFE9FFFF0EE3CFEAFF56
:10239000E9CFF3FFEACFF4FF0900F5CFEFFFEE66D8
:1023A000FBD71200FE0EE3CFE9FFFF0EE3CFEAFFFB
:1023B000F36AF46AEE5203E0F34AF42AFBD7120000
:1023C000D9CFE6FFDACFE6FFE1CFD9FFE2CFDAFFE0
:1023D000E652E652CE50DF6E010ECFCFDBFFDECFEE
:1023E00014F0DDCF15F014C0F3FF15C0F4FFE55273
:0E23F000E552E552E5CFDAFFE7CFD9FF120044
:0223FE00D9CF35
:10240000E6FFDACFE6FFE1CFD9FFE2CFDAFFE6520F
:10241000E652FC0EDBCFDEFFDBCFDDFF010EDB5033
:10242000CF6EDF50CE6EE552E552E552E5CFDAFFD2
:06243000E7CFD9FF120006
:0A243600D9CFE6FFDACFE6FFE1CFD1
:10244000D9FFE2CFDAFFE652E652FC0EDBCFDEFF29
:10245000DBCFDDFF010EDB50D76EDF50D66EE552CD
:0E246000E552E552E5CFDAFFE7CFD9FF1200D3
:02246E00D9CFC4
:10247000E6FFDACFE6FFE1CFD9FFE2CFDAFFACAC7F
:1024800004D0AC900101EAB3AC80FD0EDB50AD6E20
:0C249000E552E5CFDAFFE7CFD9FF1200DC
:04249C00000EF36ECD
:1024A00000EE00F0060E01D81200EA6002D0EE6ADB
:0C24B000FCD7F350E9601200EE6AFCD784
:0424BC0015EE00F029
:1024C00025EE00F0F86A0F9C6AEC11F003EC00F0C6
:0824D00013EC08F0FBD7120029
:0824D800FF0EE350E84E120074
:0E24E000000000D000D000D0E82EFAD7120085
:0224EE001E21AD
:1024F0002221452167218721B921F12129223A2270
:102500004B225C226D227E228F22A022B122C22287
:1025100000000000000000000000000000000000BB
:1025200000000000000000000000000000000000AB
:10253000000000000000000000000000000000009B
:10254000000000000000000000000000000000008B
:10255000000000000000000000000000000000007B
:1025600000003030303030303030003132333435EC
:102570003637383930313233343536003030303058
:10258000303030303030303030303030303030304B
:102590003030300007070707070707070707070757
:1025A00007070707070707070707070707070707BB
:1025B00007070707070707070707070707070707AB
:0E25C0000707070707070707070707070000B9
:020000040030CA
:0100010022DC
:0100020004F9
:010003000EEE
:010006008178
:00000001FF
